:020000040000FA
:1000000008288207000080293C2A4129902AE42AF6
:100010008B0109235B235908AA005A08AB005B082F
:10002000AC005C08AD0051275508AA005608AB008B
:100030005708AC005808AD003F27851400000000A9
:1000400000000000851085120430870021218516EC
:100050000000000085120030870021218516000075
:100060000000851205185D289223922305185D284B
:100070002D21FF30F800F9000930FA000518592841
:10008000F80B3E28FF30F800F90B3E28FF30F9004E
:10009000FA0B3E28FF30F800F9000930FA00F51895
:1000A0005428F1210330C200F514051C55282D21D8
:1000B0005D2892239223051C3E2889254A08E900E1
:1000C0004908EA004808EB004708EC004608ED0044
:1000D0004508EE004408EF004308F0004824650896
:1000E000DD006608DE006708DF006808E0005208EF
:1000F000E9005108EA005008EB004F08EC004E08F8
:10010000ED004D08EE004C08EF004B08F0004824CD
:100110006608E1006708E2006808E300E401F51BF7
:10012000A32886015D08F1005E08F2005F08F30075
:100130006008F40075100921051500000511013053
:10014000F600F7003228751CFC28F70B32285308FC
:10015000013A031DAE280130F700BE285308023AC9
:10016000031DB5280330F700BE285308033A031DCA
:10017000BC280830F700BE280F30F700760987004A
:10018000870A000005150000051109217108A0006B
:100190007208A1007308A2007408A3006108A400FB
:1001A0006208A5006308A6006408A7009F23200832
:1001B000F1002108F2002208F3002308F400F60BF6
:1001C0003228FF30F6002230F100F201F301F40191
:1001D000092176098700870A00000515000005112E
:1001E0005D08F1005E08F2005F08F3006008F400AB
:1001F000051600000512322875145D08F1005E082E
:10020000F2005F08F3006008F40005160000051214
:10021000A52885120030870021217408870021213C
:100220007308870021217208870021217108870047
:10023000212100000000851600000000000085124A
:10024000080000000000000085150000000000000C
:1002500085110000000000000800F5183B29751DFD
:1002600035290D2275110330C200C20B3929023025
:10027000C20042080128C20B3F290530C2004208D3
:1002800001285330B0007030B1006530B200B300C7
:100290006430B4003D30B5002030B600B700B8007F
:1002A000BD006D30BE007330BF005308013A031D1E
:1002B00061292030B9003130BA003030BB00BC00B9
:1002C000072B5308023A031D6D292030B900323044
:1002D000BA003030BB00BC00072B5308033A031DA3
:1002E00079292030B9003530BA003030BB00BC006D
:1002F000072B3130B9003030BA00BB00BC00072BEF
:100300005330B0007430B1006530B2007030B300CB
:100310003D30B4002030B500B600B700B800BC00D6
:100320004830BE007A30BF005408013A031D9F29AF
:100330002030B900BA00BD003130BB00072B540893
:10034000023A031DAB292030B900BD003130BA009C
:100350003030BB00072B5408033A031DB729313056
:10036000B9003030BA00BB002030BD00072B540864
:10037000043A031DC3292030B900BA003130BB0054
:100380006B30BD00072B5408053A031DD0292030DF
:10039000B9003130BA003030BB006B30BD00072BE4
:1003A0005408063A031DDC293130B9003030BA0058
:1003B000BB006B30BD00072B5408073A031DE8292A
:1003C0002030B900BA003130BB004D30BD00072BE2
:1003D0002030B9003130BA003030BB004D30BD00A4
:1003E000072B2030B000B100B700BC00BF00533075
:1003F000B2005730B3004530B400B500B9005030FA
:10040000B6004D30B8004E30BA00BE005530BB00CB
:100410004F30BD0007232A2208002030B000B10071
:10042000B700BC005330B2005730B3004530B400C1
:10043000B500B9005030B6004D30B8004E30BA00AB
:100440005530BB004F30BD004630BE00BF00072313
:100450002A220800FF30F800F9003230FA00F80BC9
:100460002F2AFF30F800F90B2F2AFF30F900FA0B82
:100470002F2A0930FA0008004630B0003D30B100A4
:100480002030B200BD002E30B500B9004830BE00AB
:100490007A30BF00C30803194E2A772A2030B300F0
:1004A000C4080319542A7A2A2030B400B500C508BC
:1004B00003195B2A7D2A2030B600C6080319612A79
:1004C000802A2030B700C7080319672A832A203002
:1004D000B800B900C80803196E2A862A2030BA006D
:1004E000C9080319742A892A2030BB008C2A4308C2
:1004F000303EB3004408303EB4004508303EB600FC
:100500004608303EB7004708303EB8004808303E45
:10051000BA004908303EBB004A08303EBC00072BF9
:100520004230B0003D30B1002030B200BD002E306E
:10053000B500B9004830BE007A30BF00CB080319BF
:10054000A22ACB2A2030B300CC080319A82ACE2A2D
:100550002030B400B500CD080319AF2AD12A2030CD
:10056000B600CE080319B52AD42A2030B700CF0828
:100570000319BB2AD72A2030B800B900D0080319C4
:10058000C22ADA2A2030BA00D1080319C82ADD2A83
:100590002030BB00E02A4B08303EB3004C08303E10
:1005A000B4004D08303EB6004E08303EB7004F084C
:1005B000303EB8005008303EBA005108303EBB0013
:1005C0005208303EBC00072B5330B0007730B100EA
:1005D0006530B2006530B3007030B4003D30B50016
:1005E0002030B600B700B800B900BA00BB00BC00AC
:1005F000F51F012B2030BD004F30BE004E30BF0034
:10060000072B4F30BD004630BE004630BF004223AE
:1006100008008312031385018601870183162730A2
:1006200081000130850003308600003087000C1007
:100630000C13FF309F0083121F1098139412101098
:100640001211F5100230C2000430D3000730D4007C
:10065000FF30F800F9000930FA00FF30C1004030E7
:10066000D5004B30D6004C30D7000030D800B83021
:10067000D9000B30DA000030DB000030DC00F5136D
:10068000751108000230A1008030AE0030308400C7
:100690000830AF002E087623AE0A00088023840AB3
:1006A000AF0B4A2BC030AE00383084000830AF00AA
:1006B000A10B4A2B080092239223303086008C2312
:1006C00092238C2392238C239223203086008C2328
:1006D00092232830762392230C3076239223013004
:1006E000762392230630762392230800C000F03947
:1006F00086008C23400EF03986008C23860108008A
:10070000C000F039860006158C23400EF0398600B3
:1007100006158C23860108009A2386159A238611D4
:100720009A2308001E30AF00AE01AE0B952BAF0B25
:10073000942B08001E30A000A00B9C2B080024085E
:10074000A00725080318250FA10726080318260F60
:10075000A20727080318270FA30708002408A002F0
:100760002508031C250FA1022608031C260FA20240
:100770002708031C270FA3020800230827060319D4
:10078000C52BAD0023308400DC2B2208260603197C
:10079000CD2BAD0022308400DC2B21082506031967
:1007A000D52BAD0021308400DC2B20082406031952
:1007B0000034AD0020308400AD1FE12B801F2D34AC
:1007C0002B342D1FE62B001F2D342B34AD1EEB2BAD
:1007D000801E2D342B342D1EF02B001E2D342B3477
:1007E000AD1DF52B801D2D342B342D1DFA2B001D36
:1007F0002D342B34AD1CFF2B801C2D342B34001CCE
:100800002D342B3403102030A800A001A101A20137
:10081000A301A401A501A601A701AA0DAB0DAC0D72
:10082000AD0DA00DA10DA20DA30DA80B302C230E14
:100830000F39A70023080F39A600220E0F39A50093
:1008400022080F39A400210E0F39A30021080F3907
:10085000A200200E0F39A10020080F39A0000800C7
:10086000203084003D24213084003D242230840047
:100870003D24233084003D240D2C03300007A900C3
:10088000A919800030300007A900A91B800000349E
:10089000E501E601E701E8016330A0000730A100AF
:1008A000A201A301693084001D256508A400660823
:1008B000A5006708A6006808A7009F232008E50098
:1008C0002108E6002208E7002308E8008730A0009E
:1008D0000730A100A201A3016A3084001D2565082C
:1008E000A4006608A5006708A6006808A7009F2363
:1008F0002008E5002108E6002208E7002308E800B8
:10090000AB30A0000730A100A201A3016B3084002E
:100910001D256508A4006608A5006708A6006808EC
:10092000A7009F232008E5002108E6002208E70031
:100930002308E800CF30A0000730A100A201A301E6
:100940006C3084001D256508A4006608A5006708B2
:10095000A6006808A7009F232008E5002108E600FC
:100960002208E7002308E800F330A0000730A100C8
:10097000A201A3016D3084001D256508A40066084E
:10098000A5006708A6006808A7009F232008E500C7
:100990002108E6002208E7002308E8001730A0003D
:1009A0000830A100A201A3016E3084001D25650856
:1009B000A4006608A5006708A6006808A7009F2392
:1009C0002008E5002108E6002208E7002308E800E7
:1009D0003B30A0000830A100A201A3016F308400C9
:1009E0001D256508A4006608A5006708A60068081C
:1009F000A7009F232008E5002108E6002208E70061
:100A00002308E8005F30A0000830A100A201A30184
:100A1000703084001D256508A4006608A5006708DD
:100A2000A6006808A7009F232008E5002108E6002B
:100A30002208E7002308E80008008008031D232D92
:100A4000A001A1010800800D000DA400A403A501D0
:100A5000A601A7019F232108031783128F00031308
:100A6000200803178D0083160C1400000000831269
:100A70000C080313A8000130A400A501A601A701DA
:100A8000AE23200803178D000313210803178F00DE
:100A900083160C140000000083120C080313A90035
:100AA0000130A400A501A601A701AE232008031769
:100AB0008D000313210803178F0083160C14000008
:100AC000000083120C080313AA000130A400A50142
:100AD000A601A701AE23200803178D0003132108E8
:100AE00003178F0083160C140000000083120C08FB
:100AF0000313AB000130A400A501A601A701AE239A
:100B00002808A0002908A1002A08A2002B08A30099
:100B10000800061C922D411C982D861C952DC11C89
:100B2000982D08004118982D8D2DC118982D08007A
:100B3000C10DC10D061C9E2D41149F2D4110861C18
:100B4000A32DC114A42DC1104108E13A031DA92D04
:100B5000AE2D4108D23A031D0800632E4208033A25
:100B6000031DBA2DD30A5308053A031D5529013038
:100B7000D30055294208013A031DC62DD40A540852
:100B8000093A031D94290130D40094294208023AFD
:100B9000031DFC2D5508A0005608A1005708A2000F
:100BA0005808A300EB269F23A4015930A50062300A
:100BB000A6000230A700BD232B3A031DEF2DA00194
:100BC000D501AA015930A100D600AB006230A200C5
:100BD000D700AC000230A300D800AD003F2F2008A2
:100BE000D500AA002108D600AB002208D700AC002F
:100BF0002308D800AD003F2F4208043A031D5C2EA5
:100C00005908A0005A08A1005B08A2005C08A300D4
:100C1000EB269F232008E5002108E6002208E700D4
:100C20002308E800A0015A30A1006230A20002307F
:100C3000A3005508A4005608A5005708A6005808A8
:100C4000A700AE232008A4002108A5002208A600C2
:100C50002308A7006508A0006608A1006708A20095
:100C60006808A3002408E5002508E6002608E70038
:100C70002708E800BD232B3A031D4F2E6508A0006E
:100C8000D900AA006608A100DA00AB006708A2003C
:100C9000DB00AC006808A300DC00AD00512F200889
:100CA000D900AA002108DA00AB002208DB00AC0062
:100CB0002308DC00AD00512F4208053A031D08004F
:100CC000F51FF517E42A4208033A031D6C2ED30BD7
:100CD00055290430D30055294208013A031D752EC9
:100CE000D40B94290830D40094294208023A031DF9
:100CF000AB2E5508A0005608A1005708A2005808BE
:100D0000A300EB26BD232D3A0319902EAE231430F9
:100D1000A400A501A601A701BD232D3A031D9E2E07
:100D20001430A000D500AA00A101D601AB01A20198
:100D3000D701AC01A301D801AD013F2F2008D50098
:100D4000AA002108D600AB002208D700AC00230877
:100D5000D800AD003F2F4208043A031DE12E590888
:100D6000A0005A08A1005B08A2005C08A300EB26C3
:100D7000BD232D3A0319C62EAE23FF30A400A501D2
:100D8000A601A701BD232D3A031DD42EFF30A000DC
:100D9000D900AA00A101DA01AB01A201DB01AC017B
:100DA000A301DC01AD01512F2008D900AA002108C0
:100DB000DA00AB002208DB00AC002308DC00AD0049
:100DC000512F4208053A031D0800F51FE42AF513C8
:100DD000F5107515E42A01305406031DF52E013077
:100DE000A400A501A601A701080002305406031DB6
:100DF000FF2E0A30A400A501A601A70108000330B8
:100E00005406031D092F6430A400A501A601A70103
:100E1000080004305406031D142FE830A4000330EA
:100E2000A500A601A701080005305406031D1F2FC9
:100E30001030A4002730A500A601A7010800063045
:100E40005406031D2B2FA030A4008630A5000130CE
:100E5000A600A701080007305406031D372F4030B5
:100E6000A4004230A5000F30A600A7010800803082
:100E7000A4009630A5009830A600A701080002241F
:100E80002708C3002608C4002508C5002408C6009A
:100E90002308C7002208C8002108C9002008CA008A
:100EA0003C2A02242708CB002608CC002508CD00C8
:100EB0002408CE002308CF002208D0002108D1004A
:100EC0002008D200902A000000000000220000004C
:100ED0000000000044000000000000006700000067
:100EE000000000008900000000000000AB000000CE
:100EF00000000000CE00000000000000F000000034
:100F00000000010012000000000001003500000098
:100F1000000001005700000000000200AF000000C8
:100F20000000040006000000000005005E00000054
:100F300000000600B5000000000008000D000000E1
:100F4000000009006500000000000A00BC0000006D
:100F500000000C001400000000000D006B000000F9
:100F600000001A00D7000000000028004300000025
:100F700000003500AF000000000043001B0000002F
:100F8000000050008700000000005D00F30000003A
:100F900000006B005F00000000007800CB00000044
:100FA000000086003700000001000C006F00000008
:100FB00001009200A700000002001800DE000000FF
:100FC00002009F0016000000030024005E000000E5
:100FD0000300AB008600000004003100BD000000EB
:100FE0000400B700F500000005003E002D000000E1
:100FF0000A007C005A0000000F00BA0088000000C0
:101000001400F800B50000001A003600E2000000ED
:101010001F007500100000002400B3003D00000018
:101020002900F1006B0000002F002F009800000045
:1010300034006D00C50000006800DB008B0000007C
:101040009D00490051000000D100B70017000100C9
:1010500006002400DD0001003A009200A300010018
:101060006F00000068000100A3006E002E00010068
:10107000D700DB00F40002000C004900BA000400B5
:1010800018009300740006002400DD002F00080003
:1010900031002600E9000A003D007000A3000C00AA
:1010A0004900BA005E000E0056000400180010004F
:1010B00062004D00D20012006E0097008D001400F7
:1010C0007A00E10047002800F500C2008F003D00D3
:1010D0007000A300D7005100EB0085001E005300F4
:1010E00077006500650070002000470065006E0015
:1010F00065007200610074006F00720020005A00E9
:1011000055004D00450052002000560031002E00D1
:0C111000330020003200300031003500B8
:02400E00B23FBF
:00000001FF
